:0200000480007A
:100000006F004005732F2034930F8000630AFF03B5
:10001000930F90006306FF03930FB0006302FF038A
:10002000170F0000130F0F3E63040F0067000F004F
:10003000732F203463540F006F00400093E19153FD
:10004000171F000023203FFC171F0000232E0FFA6C
:100050006FF01FFF930000001301000093010000E8
:10006000130200009302000013030000930300003A
:100070001304000093040000130500009305000022
:10008000130600009306000013070000930700000A
:1000900013080000930800001309000093090000F2
:1000A000130A0000930A0000130B0000930B0000DA
:1000B000130C0000930C0000130D0000930D0000C2
:1000C000130E0000930E0000130F0000930F0000AA
:1000D000732540F16310050097020000938202012E
:1000E000739052307350447497020000938202015F
:1000F00073905230735000189702000093820202EE
:1001000073905230B70200809382F2FF7390023BEB
:100110009302F0017390023A73504030970200004E
:1001200093824201739052307350203073503030BC
:100130009301000097020000938202ED7390523009
:10014000130510001315F501634C05000F00F00FA7
:10015000930110009308D005130500007300000000
:1001600093020000638A020073905210B7B200003D
:100170009382921073902230735000303725000024
:100180001305058073200530970200009382420119
:1001900073901234732540F17300203093012000D6
:1001A000000000006F000013B7220000938202805D
:1001B00073B0023037130000130303807320033041
:1001C000F3230030B3F353006314731273504134BC
:1001D00073504130970200009382D22273945230C0
:1001E000F322503093F212006386020073600430F1
:1001F0006F000000731054307350313097020000CC
:100200009382820273901234B7220000938202809C
:1002100073B00230371300001303038073200330E0
:100220007300203073005010B3F20200B7020C00CC
:1002300073B002103373030037030C0073200310F4
:10024000F3230010B3F353006384030673B002106A
:1002500073000012F3220018000000006F008007F6
:10026000730000126F000007F32200186F00800671
:1002700097020000938202027390121493020010FE
:1002800073A002109302000273B0021073002010DA
:10029000000000006F00000497020000938202013A
:1002A00073901214730020106F00C0026F004002A0
:1002B000730000126F000002730000126F008001D3
:1002C000F3220018000000006F00C0006FF05FFA1A
:1002D000631030020F00F00F638001009391110052
:1002E00093E111009308D00513850100730000000D
:1002F0000F00F00F930110009308D00513050000C4
:100300007300000013000000130000001300000041
:100310001300000013000000130000001300000091
:100320001300000013000000130000001300000081
:100330001300000013000000130000001300000071
:100340001300000013000000130000001300000061
:100350001300000013000000130000001300000051
:100360001300000013000000130000001300000041
:100370001300000013000000130000001300000031
:100380001300000013000000130000001300000021
:100390001300000013000000130000001300000011
:1003A0001300000013000000130000001300000001
:1003B00013000000130000001300000013000000F1
:1003C00013000000130000001300000013000000E1
:1003D00013000000130000001300000013000000D1
:1003E00013000000130000001300000013000000C1
:1003F00013000000130000001300000013000000B1
:100400006F0000046FF01FDF6FF0DFEC6FF09FEC08
:100410006FF05FEC6FF01FEC6FF0DFEB6FF09FEBB6
:100420006FF05FEB6FF01FEB6FF0DFEA6FF09FEAAA
:100430006FF05FEA6FF01FEA6FF0DFE96FF09FE99E
:1004400013032000F3222034E39662E8F3221034F1
:10045000F3233034638E030003D30200B3C363007D
:1004600003D3220013130301B3C36300E39403E631
:1004700017030000130303D363846206170300000D
:100480001303C3DD6384620617030000130383DDD7
:100490006388620417030000130343DD6382620470
:1004A00017030000130303DF6388620417030000CF
:1004B000130383DF6388620417030000130383DFE1
:1004C0006386620217030000130343DF638A62003E
:1004D00017030000130343DF638462006FF09FDFA4
:1004E000938282007390123473002030370310001F
:1004F000732003306FF0DFFE3703400073200330BA
:100500006FF01FFE6FF0DFFD731000C000000000F1
:1005100000000000000000000000000000000000DB
:1005200000000000000000000000000000000000CB
:1005300000000000000000000000000000000000BB
:1005400000000000000000000000000000000000AB
:10055000000000000000000000000000000000009B
:10056000000000000000000000000000000000008B
:10057000000000000000000000000000000000007B
:10058000000000000000000000000000000000006B
:10059000000000000000000000000000000000005B
:1005A000000000000000000000000000000000004B
:1005B000000000000000000000000000000000003B
:1010000000000000000000000000000000000000E0
:1010100000000000000000000000000000000000D0
:1010200000000000000000000000000000000000C0
:1010300000000000000000000000000000000000B0
:081040000000000000000000A8
:040000058000000077
:00000001FF
